:1000000064C17DC17CC17BC17AC179C178C177C12E
:1000100076C175C174C173C172C171C170C16FC144
:100020006EC16DC16CC11600170019001B001E00C7
:10003000220027002D0034003D00490058006A00CE
:1000400082009F00C400F3002E017801D5014A020E
:10005000DE029703FFFF1500160018001A001C00AF
:100060001F00230028002E00360040004C005C00DA
:100070006F008800A600CC00FB0036017F01D8018C
:100080004502C9026703FFFF0300040005000600E4
:10009000070009000B000E00120016001C002300D0
:1000A0002C00370044005500690081009E00C2000A
:1000B000EC001E015A019F01F1015002C0024103F0
:1000C000D703FFFF0400060007000A000C00100021
:1000D000130018001D0023002A0033003C004700D5
:1000E00053006200720085009B00B300D000F00056
:1000F00014013E016D01A201E00124027F022C03E4
:10010000FFFF5072652D417474656E756174696F7F
:100110006E207365743A203A78782E78782064429D
:1001200020207573652052656C2D526573657420AF
:100130002620205A65726F2D41646A20746F2073E7
:100140006574005741524E494E47204F5645524C18
:100150004F4144202072656475636520696E707537
:1001600074202020706F77657220746F2061766F25
:1001700069642064616D616765206F662073656ED8
:10018000736F72004261747465727920566F6C747B
:1001900061676520202020202D2E2D20566F6C7445
:1001A0007320202020205374617475733A202D6FC2
:1001B0006F2D2020202020202020202020202020E3
:1001C0002020202000546865726D616C2D53656E8F
:1001D000732E7820206162733A203A78782E7878EE
:1001E0002064426D2072656C3A203A78782E7878D7
:1001F0002064422020202020202020202020202099
:1002000020202020200044696F64652D53656E73A3
:100210006F72202020206162733A203A78782E781D
:10022000782064426D2072656C3A203A78782E7896
:100230007820644220202078787878202073656EBA
:10024000736F72202D200020204144432D7261776E
:1002500076616C75652020666F722063616C6962DF
:10026000726174696F6E20414430204144312041F5
:10027000443220414434202D2D2D202D2D2D202D94
:100280002D2D202D2D2D200020204475616C2D5307
:10029000656E736F7220202020524620506F776564
:1002A000726D6574657220204453504D30332020A8
:1002B0005665727320322E30286329203230303553
:1002C0002020444C354E4547000011241FBECFE589
:1002D000D4E0DEBFCDBF10E0A0E6B0E0E6E5FEE092
:1002E00002C005900D92A436B107D9F710E0A4E63C
:1002F000B0E001C01D92A23BB107E1F704C380CE7C
:10030000AF92BF92CF92DF92EF92FF920F931F9323
:10031000CF93DF93282F332742E7A42E40E0B42E5B
:1003200093E4C92E91E0D92E84E8E82E81E0F82EDE
:1003300005EC11E0C2E0D1E0A6E0B2E067E472E0D3
:1003400048E852E09FE32430310501F125303105C2
:1003500054F422303105A1F023303105A4F42130CA
:10036000310559F020C026303105B1F02630310575
:1003700084F02730310599F016C0FA01849111C03C
:10038000FB0184910EC0FD0184910BC0FE0184919C
:1003900008C0F801849105C0F701849102C0F601FC
:1003A0008491F501808391504F5F5F4F6F5F7F4F66
:1003B000119621960F5F1F4F0894E11CF11C0894C1
:1003C000C11CD11C0894A11CB11C97FFBCCFDF91AC
:1003D000CF911F910F91FF90EF90DF90CF90BF9042
:1003E000AF900895982F12BE83E083BF992341F008
:1003F00008B600FEFBCF915088B7816088BFF6CF6A
:1004000008951F93CF93DF93982F86EE86B997B9FF
:10041000C0E0D0E01FE081E0E5DF24B185B199279D
:10042000982F8827820F911DC80FD91F115017FFD1
:10043000F2CFCE0154E0969587955A95E1F7DF917A
:10044000CF911F91089520916200233009F580918A
:100450006000882359F081E68093A30085E78093AC
:10046000A40084E78093A5008FE60AC08DE6809300
:10047000A30081E68093A4008EE68093A50080E22D
:100480008093A60080916100805D8093B0000BC0D6
:10049000253049F480916A00882311F481E301C07A
:1004A00082E380937F0080E280938100233011F00B
:1004B000253049F48091680090916900892B19F0EA
:1004C00081E480938100223011F0253039F480914D
:1004D0006700882319F08AE58093810008950895C4
:1004E000805D8A3308F0895F992708954F925F9263
:1004F0006F927F928F929F92AF92BF92CF92DF9234
:10050000EF92FF920F931F93CF93DF9300916800B8
:1005100010916900EC01C00FD11FD0936F00C09300
:100520006E0080E070906200C0907000D09071000A
:10053000409087005090880060908900F0918B0077
:10054000A0918C00E0906400F0906500809097008E
:1005500090909800A0909900B0909B0090919C0082
:100560009E0144E0741611F4980104C0882311F030
:100570002C193D0937FF05C0309521953F4FBDE24D
:1005800001C0BBE240E050E0E0E02417350724F072
:1005900048515C4FEF5FF9CFE150241B350B2851D8
:1005A0003C4F40E050E070E02417350724F04C59F0
:1005B0005F4F7F5FF9CF7150241B350B2C593F4F94
:1005C00040E050E060E02417350724F0465F5F4FBD
:1005D0006F5FF9CF6150241B350B265F882319F01C
:1005E00034E0731689F44B2E40E3542E5E0E30E354
:1005F000632E670EF62FF05DA22FA05DE114F104CB
:1006000079F0FFE5AF2F0CC08B2EB0E39B2E9E0E32
:10061000E0E3AE2EA70E70E3B72EB60E922F905DDC
:100620008F5F823008F49CCF90939C00B0929B0027
:10063000A09299009092980080929700A0938C00CD
:10064000F0938B006092890050928800409287005E
:10065000DF91CF911F910F91FF90EF90DF90CF909E
:10066000BF90AF909F908F907F906F905F904F90D2
:100670000895FC013196849131979927982F882706
:100680002491820F911D0895BF92CF92DF92EF9235
:10069000FF920F931F93CF93DF937C01BB24C0E0A5
:1006A000D0E08E016E01809162002ADECCDEB09235
:1006B0006B00809162008330B1F5809161008130E0
:1006C000D1F401C0B394CB2DDD27CC0FDD1F8E01FB
:1006D0000C531F4FC801CDDFE816F90698F7F2EF6B
:1006E000CF2EFFEFDF2EC801C4DF8C01CE018E5369
:1006F0009F4F17C0B394CB2DDD27CC0FDD1F8E018C
:1007000008571F4FC801B5DFE816F90698F7E2EE63
:10071000CE2EEFEFDE2EC801ACDF8C01CE018A5762
:100720009F4FA7DFEC01809162008530C9F5809171
:100730006A008823D1F4B82E01C0B394CB2DDD27F5
:10074000CC0FDD1F8E010A5A1F4FC80192DFE81639
:10075000F90698F77DEFC72E7FEFD72EC80189DF06
:100760008C01CE018C5A9F4F19C0BB2401C0B39499
:10077000CB2DDD27CC0FDD1F8E010A5D1F4FC80179
:1007800078DFE816F90698F766EFC62E6FEFD62EDB
:10079000C8016FDF8C01CE018C5D9F4F6ADFEC01D9
:1007A000BB2081F48CE3809386008093960084E6DE
:1007B00090E0C89E9001C99E300DD89E300D112446
:1007C000C90126C03FEF0F3F130731F487E098DDE2
:1007D00081E080936B001DC00C1B1D0BEC1AFD0A01
:1007E000E4E6F0E0EE9EC001EF9E900DFE9E900DBF
:1007F0001124B80109D3CB0CD11CCE9EC001CF9ED1
:10080000900DDE9E900D1124860F971F8456904008
:100810006DDEDF91CF911F910F91FF90EF90DF90F0
:10082000CF90BF900895009711F00197FCCF0895E5
:10083000089582BBC29AC29882E390E0F4DF0895E3
:100840000F931F93CF93AD9880E8F3DF84E0CADD68
:10085000AD9A02E710E0CFE0F80181918F01E9DF66
:10086000C150C7FFF9CF02E910E0CFE0F801819154
:100870008F01DFDFC150C7FFF9CFAD9880ECD9DF22
:1008800084E0B0DDAD9A02E810E0CFE0F80181919C
:100890008F01CFDFC150C7FFF9CF02EA10E0CFE0F0
:1008A000F80181918F01C5DFC150C7FFF9CFCF910A
:1008B0001F910F9108958091620022DDC1DF89E1CF
:1008C00091DD0895CF938AE08DDD85B38F7C85BB64
:1008D000C2E080E3AEDF81E085DDC150C7FFF9CF24
:1008E000C4E088E3A6DF81E07DDD8CE0A2DF81E06B
:1008F00079DD81E09EDF8C2F75DD82E09ADF8C2F21
:1009000071DDCF910895CFE5D4E0DEBFCDBF1FEFFD
:1009100011BB80E284BB86E087BB89E388BB83E8A8
:100920008FBD01E00EBD80E092E090936D0080935A
:100930006C0082E08BBD80916C008ABDC3DF802F8C
:10094000DFDC7EDF812F4EDD812F4CDD812F4ADD04
:1009500083E080936200D4DC73DF8091670088239A
:1009600069F180916A004DDD8C01809167008130D2
:1009700029F40031110510F0109267008091670092
:100980008F3F29F40131110510F410926700809116
:100990006700282F332727FD309580916C009091B8
:1009A0006D00820F931F90936D0080936C00892FD0
:1009B000990F990B8BBD80916C008ABD86B3082F6F
:1009C000112703FF0FC005FF0DC010926600809134
:1009D000640090916500009729F00197909365005D
:1009E0008093640000FD0BC0809162008F5F809354
:1009F0006200873018F082E0809362005CDF04FDC3
:100A000026C0809162008330A9F48091600081301B
:100A100019F41092600005C080916100813021F4CA
:100A20008F5F8093610012C081E0809361008093AA
:100A300060000CC0853051F480916A00882319F061
:100A400010926A0003C084E080936A0034DF03FDE3
:100A50004FC080916200843009F041C080916800ED
:100A60009091690027E1803792070CF041C09C010A
:100A70002F5F3F4F3093690020936800909166008C
:100A8000892F8F5F809366008A3040F090936600D4
:100A900082E390E09093650080936400809164000D
:100AA00090916500892BC1F0C90164E670E0ACD17A
:100AB000892B61F02F5F3F4FC90164E670E0A4D13C
:100AC000892BC1F7309369002093680082E390E09E
:100AD00090936500809364008EE184DC09C080916E
:100AE0006E0090916F009093710080937000E3DE30
:100AF00005FD5DC080916200823011F0853099F46F
:100B000080916700882379F480916A007ADC8C01F7
:100B1000419718F08FEF809367000031110518F4AA
:100B200081E08093670080916200843009F03FC0CB
:100B3000809168009091690028EE81399207BCF19C
:100B40009C012150304030936900209368009091BF
:100B50006600892F8F5F809366008A3040F0909303
:100B6000660082E390E0909365008093640080913A
:100B7000640090916500892BC1F0C90164E670E0C2
:100B800043D1892B61F021503040C90164E670E007
:100B90003BD1892BC1F7309369002093680082E331
:100BA00090E090936500809364008EE11BDC80915F
:100BB000620099278430910509F49BC08530910526
:100BC0003CF48230910561F0039709F477C0C4CEFC
:100BD0008530910509F491C0069709F4E3C0BCCEB5
:100BE00032DC80E00EDC8C018F707ADC8093A40014
:100BF00064E0169507956A95E1F7802F8F7070DC99
:100C00008093A30054E0169507955A95E1F7802F3D
:100C10008F7066DC8093A20081E0F3DB8C018F7023
:100C20005FDC8093A80044E0169507954A95E1F7AC
:100C3000802F8F7055DC8093A70034E016950795C0
:100C40003A95E1F7802F8F704BDC8093A60082E00D
:100C5000D8DB8C018F7044DC8093AC0024E01695C7
:100C600007952A95E1F7802F8F703ADC8093AB00CF
:100C700094E0169507959A95E1F7802F8F7030DCF8
:100C80008093AA0084E0BDDB8C018F7029DC809307
:100C9000B00084E0169507958A95E1F7802F8F7054
:100CA0001FDC8093AF00B4E016950795BA95E1F785
:100CB000802F8F7015DC8093AE004ECE8091610046
:100CC000A0DB8C0180916000882381F00332110544
:100CD00018F482E080936100085D134018F081E011
:100CE00080936100809161008CDB8C01C801CCDCB9
:100CF00033CE80E090E0FADB2FCE80916A0081DB7A
:100D00008C01C2DC80916B00813009F425CE00316A
:100D1000110539F48CE38093A9008EE38093AA0037
:100D20001BCE01311105F8F09801295D3F4F2034A9
:100D3000310514F02FE330E0F901EE58FF4F8EE358
:100D4000808347E3283331050CF406CE5DE2E42FBF
:100D5000FF27EE58FF4F50834F5F842F992782174C
:100D60009307ACF3F9CD9801285D3F4F203331054F
:100D700014F420E330E0F901EE58FF4F8CE3808358
:100D800048E3283331050CF0E7CD5DE2E42FFF277F
:100D9000EE58FF4F50834150842F99272817390769
:100DA000ACF3DACD83E02DDB8C018158924028F042
:100DB00084E680939F0087E604C082E780939F00CB
:100DC00080E780939C00A3E016950795AA95E1F72C
:100DD00080E090E020E00A962F5F08171907D8F707
:100DE0002150081B190BE02FE65F2A3018F02A501B
:100DF00081E301C080E280938500205D209386001E
:100E0000E05DE0938800A8CD97FB092E07260AD065
:100E100077FD04D00CD006D000201AF470956195AF
:100E20007F4F0895F6F7909581959F4F0895AA1BDF
:100E3000BB1B51E107C0AA1FBB1FA617B70710F0C5
:100E4000A61BB70B881F991F5A95A9F780959095F7
:060E5000BC01CD01089574
:040E56000101010095
:00000001FF
